:2000000022C03AC039C038C038C036C035C034C033C032C031C030C02FC02EC02DC02CC0C0
:200020002BC02AC029C040C14BC151C158C161C169C171C177C192C19DC1A5C1ADC1B4C11A
:20004000BBC1C2C1C9C111241FBECFEDCDBF10E0A0E6B0E0EAE5F7E002C005900D92A23643
:20006000B107D9F720E0A2E6B0E001C01D92A93BB207E1F7E4D26FC3C3CF1F920F920FB66A
:200080000F9211242F933F934F935F936F937F938F939F93AF93EF93FF938091B8008F5FAD
:2000A0008093B8008032A9F48091B7008F5F66E012D39093B70018BA81E090E00090B70081
:2000C00002C0880F991F0A94E2F7809582BB1092B800809162004091B700A091B80090E098
:2000E0006AE270E0E7D29C01842F90E067E070E0E1D2A901480F591F20E030E090E061E067
:2001000070E0F901E40FF51FED59FF4F8081A81738F4FB01022E01C0EE0F0A94EAF79E2BDC
:200120002F5F3F4F2730310561F798BBFF91EF91AF919F918F917F916F915F914F913F911B
:200140002F910F900FBE0F901F9018958091600090E0019681709927809360008091620069
:2001600090E00196817099278093620008956F927F928F929F92AF92BF92CF92DF92EF926C
:20018000FF920F931F93CF93DF93862E611102C0912C02C03AE2932EC82ED12CE601A99649
:2001A00086010095109590E2E92EF12C27E0722EE92D092C000CFF0B882021F0E017F10728
:2001C0002CF453C0CE17DF070CF44FC0A0906000B12C20E030E0422F882021F02E173F07E0
:2001E00024F41BC0E217F307C4F0B9016E1B7F0B77FF03C0719561957109062E000C770B27
:200200006C157D0554F4660F771F660F771F6F5F7F4FC70179D2662E01C0612C842F672DA5
:200220005AD2492F90E067E070E044D2DC01C5016AE270E03FD28A0F9B1FDC01AD59BF4F69
:20024000A40FB11D6C922F5F3F4F2A32310519F67DDF8FE39CE90197F1F700C00000882027
:2002600011F09A94A5CF9394A3CFDF91CF911F910F91FF90EF90DF90CF90BF90AF909F9089
:200280008F907F906F900895262F90E08830910508F053C0FC01ED5EFF4F8091600090E0FF
:2002A0006AE270E007D20994FC01ED59FF4F228323832483258326832783208721870895C2
:2002C000FC01ED59FF4F21832287278F0895FC01ED59FF4F2083268F20A323870895FC01FD
:2002E000ED59FF4F238F248F258F21A3248721A70895FC01ED59FF4F228F20A727A322A3E5
:2003000025870895FC01ED59FF4F218F26A323A324A326870895FC01ED59FF4F208F25A3AB
:2003200027870895FC01ED59FF4F208B218B228B238B248B258B268B278B0895262F90E00B
:200340008830910508F053C0FC01E55EFF4F8091600090E06AE270E0ADD10994FC01ED59DB
:20036000FF4F2187228723872487258726872787208B0895FC01ED59FF4F208721A322A379
:2003800023A3218B0895FC01ED59FF4F278320A321A724A3228B0895FC01ED59FF4F26833D
:2003A000278F25A3238B0895FC01ED59FF4F2583268F26A3248B0895FC01ED59FF4F248339
:2003C000258F27A3258B0895FC01ED59FF4F2383248F20A7268B0895FC01ED59FF4F20831F
:2003E00021832283278B208F218F228F238F08957F928F929F92AF92BF92CF92DF92EF925B
:20040000FF920F931F93CF93DF93762E942E91E0A92EA81A36E0832E880E411102C0BA2C5C
:2004200001C0B82C082F10E020E2E22EF12C992009F445C0BA140CF445C0C0E0D0E0CB2CEC
:200440000B2C000CDD08B6016C1B7D0B77FF03C0719561957109062E000C770B772081F035
:20046000601771074CF4660F771F660F771F6F5F7F4FC70149D101C060E08C2F05DF0FC04A
:20048000601771074CF4660F771F660F771F6F5F7F4FC70139D101C060E08C2F4FDF219608
:2004A000C830D10581F652DE8FE59AEE0197F1F700C00000992011F0BA94B9CFB3948B1415
:2004C0000CF0BBCFDF91CF911F910F91FF90EF90DF90CF90BF90AF909F908F907F90089512
:2004E0001F93CF93DF93A0916000B0E040E0D7E0842F6D2FFCD0C92F082E000C990B67E03E
:2005000070E0D8D09C01CD016AE270E0D3D0820F931FFC01ED59FF4FEC0FF11DC7FDFA9509
:2005200010824F5F4A3221F711DE2FEF80E792E0215080409040E1F700C00000A0916000D7
:20054000B0E040E017E0C0E2842F612FD0D0D92F082E000C990B67E070E0ACD09C01CD0103
:200560006AE270E0A7D0820F931FFC01ED59FF4FED0FF11DD7FDFA95C0834F5F4A3221F7A2
:20058000E5DD2FEF80E792E0215080409040E1F700C00000DF91CF911F910895BF92CF923A
:2005A000DF92EF92FF920F931F93CF93DF93E12CF12C0AE210E087E0B82EC0906000D12C90
:2005C000C0E0D0E0CE018E0D9F1DB8019DD06B2D82D0492F90E067E070E06CD09C01C60176
:2005E0006AE270E067D0820F931FFC01ED59FF4FE40FF11D8C2F8370880F880F880F8083DD
:200600002196CA32D105F1F6A1DD2FEF80E792E0215080409040E1F700C000002FEFE21A42
:20062000F20A84E0E816F10441F6DF91CF911F910F91FF90EF90DF90CF90BF9008951BBA73
:2006400083E08ABB9FE797BB80E888BB2FE321BB92BB86BD16BC8EB588608EBD89B7806485
:2006600089BF789488E090E09BBD8ABD8EB583608EBDC1E060E08C2F7ADD61E08C2F77DDFB
:20068000CE5FC930B9F7D1E0C1E040E06D2F8C2FAFDE41E06D2F8C2FABDECF5FC730A9F768
:2006A000D15090F71DDF1CDF1BDFC8E077DFC150E9F7DFCF0024552704C0080E591F880F7B
:2006C000991F009729F076956795B8F37105B9F7802D952F0895991B79E004C0991F961796
:2006E00008F0961B881F7A95C9F78095089587FB082E062687FD819567FD6195ECDF0EF484
:20070000919507FC8195089597FB072E16F4009406D077FD08D00BD007FC05D03EF490956C
:2007200081959F4F0895709561957F4F0895AA1BBB1B51E107C0AA1FBB1FA617B70710F000
:1C074000A61BB70B881F991F5A95A9F780959095BC01CD010895F894FFCF01006F
:00000001FF
